:100000000C94E4000C940C010C940C010C940C0165
:100010000C940C010C940C010C940C010C940C012C
:100020000C940C010C940C010C9419020C948B028E
:100030000C940C010C940C010C940C010C940C010C
:100040000C940C010C940C010C940C010C940C01FC
:100050000C940C010C940C010C940C010C94CF0129
:100060000C940C010C940C010C940C010C940C01DC
:100070000C940C010C940C010C940C010C940C01CC
:100080000C940C010C940C010C940C010C940C01BC
:100090000C94D0070C940C010C940C010C940C01E2
:1000A0000C940C010C940C010C940C01150B180B06
:1000B000070B0B0B110B390B390B390B1C0B200BDE
:1000C000240B2A0B2E0B390B340B080B00020202F7
:1000D00001000904000001020200000524001001D3
:1000E0000524010101042402060524060001070578
:1000F000810310004009040100020A000000070506
:1001000002024000000705830240000004030904C6
:1001100012010002EF02014041233680000101027A
:10012000030141726475696E6F204C4C430041724B
:100130006475696E6F204C656F6E6172646F00004C
:10014000000000240027002A002D003000000000DD
:1001500000250028002B002E0031000000000023A5
:1001600000260029002C002F0004040404040304CA
:100170000502020202040302020202060606060645
:100180000604040202020404040802011040804034
:1001900010204080408008020401804020100201AD
:1001A000108010204040200000000200090F0000D5
:1001B000030401000C00000000000000000000002B
:1001C000000000000000121211241FBECFEFDAE081
:1001D000DEBFCDBF12E0A0E0B1E0ECECFAE202C07D
:1001E00005900D92A838B107D9F724E0A8E8B2E04D
:1001F00001C01D92AF35B207E1F710E0C4EED0E0C8
:1002000004C02197FE010E945915C33ED107C9F7CA
:100210000E94440F0C9464150C9400000E945F151A
:10022000DF92EF92FF920F931F93CF93DF93D82E1D
:10023000F92EE42E062F10E0C8010196880F0E94C7
:10024000950783E00E949507CD2DDF2D0C0F1D1F14
:10025000C017D10789F0E7FE03C0FE01849101C0F9
:1002600088810E949507F82E80E00E9495078F21D3
:1002700021968111EDCF01C081E0DF91CF911F91D7
:100280000F91FF90EF90DF900895DF92EF92FF9231
:100290000F931F93CF93DF93D82E8A017B01E40E37
:1002A000F51EEB01CE15DF0571F0D7FE03C0FE0190
:1002B000849101C088810E94950721968111F2CF17
:1002C0008FEF9FEF01C0C801DF91CF911F910F9178
:1002D000FF90EF90DF9008950F931F93CF93DF93DC
:1002E0001F92CDB7DEB782E0898342E450E06AEC2A
:1002F00070E080E80E9445010E94160DDC01129614
:100300000D911C9113970115110589F0D801ED91FC
:10031000FC910280F381E02DBE016F5F7F4FC80129
:10032000099597FD04C0F80100851185ECCF8981FE
:100330000F90DF91CF911F910F9108953FB7F894DF
:100340008091A0029091A102A091A202B091A3027B
:1003500026B5A89B05C02F3F19F00196A11DB11D20
:100360003FBFBA2FA92F982F8827820F911DA11D5B
:10037000B11DBC01CD0142E0660F771F881F991F98
:100380004A95D1F708952FB7F89460919C02709127
:100390009D0280919E0290919F022FBF08951F920F
:1003A0000F920FB60F9211242F933F938F939F9329
:1003B000AF93BF9380919C0290919D02A0919E0269
:1003C000B0919F0230919B0223E0230F2D3720F440
:1003D0000196A11DB11D05C026E8230F0296A11D9F
:1003E000B11D20939B0280939C0290939D02A09349
:1003F0009E02B0939F028091A0029091A102A091D1
:10040000A202B091A3020196A11DB11D8093A0028A
:100410009093A102A093A202B093A302BF91AF91C7
:100420009F918F913F912F910F900FBE0F901F9032
:1004300018951F920F920FB60F9211248F939F93CE
:100440008091E1009091E100937F9093E10083FF20
:100450000FC01092E90091E09093EB001092EC0035
:1004600092E39093ED0010920A0398E09093F000CD
:1004700082FF20C093E09093E9009091F2009923CD
:1004800019F09AE39093E80090918C02992339F047
:1004900090918C02915090938C02992389F19091C4
:1004A0000903992339F0909109039150909309031E
:1004B000992341F184FF10C08091E2008E7E81601B
:1004C0008093E2008091E1008F7E8093E100809133
:1004D0008D028E7E806111C080FF16C08091E20087
:1004E0008E7E80618093E2008091E1008E7E809319
:1004F000E10080918D028E7E816080938D0204C028
:100500005D9ACDCF289AD6CF9F918F910F900FBE35
:100510000F901F9018951F920F920FB60F921124F3
:10052000CF92DF92EF92FF920F931F932F933F93FF
:100530004F935F936F937F938F939F93AF93BF93EB
:10054000EF93FF93CF93DF93CDB7DEB76C97DEBF0A
:10055000CDBF1092E9008091E80083FFFBC168E005
:10056000CE0145960E94C30782EF8093E8008D89F3
:1005700087FF05C09091E80090FFFCCF03C09EEF7D
:100580009093E800982F907609F0C6C09E894F8915
:10059000588D2F89F88C91110CC0803829F48091E6
:1005A00096028093F10002C01092F1001092F100C7
:1005B00045C1913051F4811141C14130510509F0DB
:1005C0003DC1809196028D7F0BC0933061F4811103
:1005D00035C14130510509F031C1809196028260E8
:1005E000809396022BC1953049F48091E80080FFFA
:1005F000FCCF822F80688093E30020C1963009F001
:100600005EC00B8D1C8D22E01092E90010928B02CF
:1006100010928A02F21232C010928902109288025D
:100620000E946C0199E0BE016F5F7F4FDB01E92FF3
:100630001D92EA95E9F79983FA8291E09E8390EA08
:1006400098879AEF998720918A0230918B02275FD1
:100650003F4F3C832B838D831092E90010928B02D5
:1006600010928A02109389020093880249E050E0B8
:1006700080E00E9445010E946C01E0C01093890255
:10068000009388020E94160DDC0112960D911C91B8
:1006900013970115110509F4BBC0D801ED91FC9128
:1006A0000480F581E02DBE016B5E7F4FC801099586
:1006B000009709F0C7C0F80100851185EACF97308F
:1006C00009F445C1983021F481E08093F100B6C06F
:1006D000993009F0B3C0837009F039C1E5E2F1E067
:1006E00081E031E096E32081211109C08EE78093FB
:1006F000EA001092EA008F8980930A039FC08093DA
:10070000E9003093EB0021912093EC009093ED00F1
:100710008F5F873041F7EACF8B8D9C8D1092E90077
:1007200010928B0210928A02909389028093880221
:10073000898D811153C08E899D89913A49F4813206
:1007400009F005C147E050E064E071E080E0BBC023
:10075000913209F0FCC0833269F48F89988DA0E052
:10076000B0E08093000190930101A0930201B09347
:10077000030164C0803269F48091E80082FFFCCFFD
:1007800067E084E091E00E94C3078BEF8093E8006C
:1007900055C0823209F052C08F8980930B01EEEF71
:1007A000FFE7859194918B3F9C4D19F0E0E0F8E0D4
:1007B00002C0EEEFFAE08091040190910501A09152
:1007C0000601B0910701803B9440A105B10509F0F5
:1007D0009EC080910B0180FF79C099C00E94160DC8
:1007E000FC01028113810115110509F4B0C0D80183
:1007F000ED91FC910190F081E02DBE016B5E7F4F89
:10080000C801099581111AC0F80100851185EBCF47
:10081000F1E0FF1609F44EC0F3E0FF1298C08F8993
:10082000882309F44AC0823089F440E860E18EE20E
:1008300091E00E941001882309F489C08EEF809313
:10084000E80088C018161906CCF381C0813029F45D
:1008500040E86BE082E291E0ECCF833009F077C0B2
:100860000E94160DDC011296ED90FC9013978E01FC
:100870000F5F1F4F6801E114F10479F0D701ED918A
:10088000FC910680F781E02DB801C7010995080F9A
:10089000111DF701E084F184EECFD8011C92F6011E
:1008A00001900020E9F73197BF016C197D0940E004
:1008B000C601BFCF60E171E002C06CE071E0FB01F6
:1008C000449150E080E80E944501B8CFEE3F2AE015
:1008D000F20751F0808191818737A7E79A0721F0CD
:1008E0009093FF0A8093FE0A87E797E791838083BE
:1008F00080916000809395029BE088E10FB6F894A8
:10090000A895809360000FBE9093600097CF808180
:1009100091818737974709F091CFA8958091600022
:100920008861809360008091950280936000EE3F23
:10093000BAE0FB0739F08091FE0A9091FF0A91839B
:1009400080837CCF1092FF0A1092FE0A77CF81E25B
:100950008093EB006C960FB6F894DEBF0FBECDBF50
:10096000DF91CF91FF91EF91BF91AF919F918F91C7
:100970007F916F915F914F913F912F911F910F91B7
:10098000FF90EF90DF90CF900F900FBE0F901F90D1
:100990001895CF92DF92EF92FF920F931F93CF9310
:1009A000DF936C017A018B01C0E0D0E0CE15DF054A
:1009B00081F0D8016D918D01D601ED91FC910190EE
:1009C000F081E02DC6010995892B11F02196EECF1B
:1009D0007E01C701DF91CF911F910F91FF90EF90A2
:1009E000DF90CF900895CF93DF931F92CDB7DEB7FE
:1009F0006983DC01ED91FC910280F381E02D41E0FF
:100A000050E0BE016F5F7F4F09950F90DF91CF914E
:100A1000089583E08093E9008091F200882319F023
:100A20008AE38093E8000895FC018485958597FD0D
:100A30000BC09FB7F89482E08093E9008091F200A8
:100A40009FBF90E0019608959FB7F89482E080934D
:100A5000E9008091F2009FBF90E0089585ED8093BA
:100A6000BC008091BC0084FDFCCF10923D03089532
:100A70004091E602262F30E0240F311D213231054E
:100A8000DCF420913D032430C9F4FC0180E090E0C7
:100A9000861758F43091E6022191DC01AA53BD4F2C
:100AA000A30FB11D2C930196F3CF8091E602680F3E
:100AB0006093E60280E0089581E0089582E0089561
:100AC0000895E091C5028091C402E81730F4F0E087
:100AD000EC55FD4F808190E008958FEF9FEF0895D2
:100AE0009091C5028091C402981750F4E92FF0E06C
:100AF000EC55FD4F208130E09F5F9093C50202C00E
:100B00002FEF3FEFC90108958091C40290E020913A
:100B1000C502821B91090895CF92DF92EF92FF9256
:100B20000F931F93CF93DF937C01CB018A01209118
:100B30003E03222389F0EB016B01C40ED51ECC15B8
:100B4000DD0569F06991D701ED91FC910190F0818B
:100B5000E02DC7010995F3CF642F0E943805C80125
:100B6000DF91CF911F910F91FF90EF90DF90CF9089
:100B70000895CF93DF931F92CDB7DEB7698320919D
:100B80003E032223D1F020916103203240F021E086
:100B900030E0FC013383228380E090E015C0809137
:100BA0003F03E82FF0E0E05CFC4F998190838F5F7A
:100BB00080933F038093610305C061E0CE010196FD
:100BC0000E94380581E090E00F90DF91CF91089569
:100BD000089580E090E008958F929F92AF92BF9227
:100BE000CF92DF92EF92FF920F931F93CF93DF93F9
:100BF0006C017B018A0180910B01882309F45CC0A0
:100C000080910A03882309F457C080918D0280FFE8
:100C100005C08091E00082608093E000E801B12C83
:100C20008AEFA82E93E0892E2AE3922E209711F4C2
:100C3000BB20D9F10E94050D81110AC0AA94AA20F7
:100C4000D9F161E070E080E090E00E940A0FEECF01
:100C5000282F30E0C217D3070CF48C2F9FB7F894DD
:100C60008092E9002091E80025FF1DC0282F30E088
:100C7000C21BD30BF701815020F041914093F1004A
:100C8000FACFE20EF31EBB2019F09092E8000AC0E2
:100C90008091E80085FD07C09092E800BB24B394E2
:100CA000209709F0B12C9FBFC1CF5D9884E6809357
:100CB0008C021016110644F081E090E0F601938357
:100CC000828380E090E001C0C801DF91CF911F9145
:100CD0000F91FF90EF90DF90CF90BF90AF909F90DB
:100CE0008F9008950E94050D90E008950F931F9333
:100CF000CF93DF931F92CDB7DEB78C01FC018485C3
:100D0000958597FF0EC0CE0101960E94D70C0197E2
:100D100019F4898190E002C08FEF9FEFF801958769
:100D20008487F801848595850F90DF91CF911F917D
:100D30000F910895CF93DF931F92CDB7DEB7FC01DB
:100D40008485958597FD05C02FEF3FEF3587248774
:100D50000BC0CE0101960E94D70C019719F489812E
:100D600090E002C08FEF9FEF0F90DF91CF91089539
:100D7000862F0C942A0D862F642F0C94530D862FEA
:100D8000642F0C94820DCF92DF92EF92FF92CF935B
:100D9000DF932091DD033091DE032130310509F02E
:100DA000BDC0C82F85E092E00E947A0C6C2F82E6CD
:100DB00093E00E94F3048DE092E00E945A0C6EEFE3
:100DC00082E693E00E94F3046AE070E080E090E045
:100DD0000E940A0FCA3209F442C01CF4C33239F02F
:100DE0009DC080ED8C0F8A3008F473C097C080E1FD
:100DF00092E00E947A0C0E947C0C81118FC0C12C61
:100E0000D12C760161E089E00E94530D68EC70E01E
:100E100080E090E00E940A0F60E089E00E94530D9C
:100E200068EC70E080E090E00E940A0F4AE0C701A1
:100E3000B6010E94960C8FEFC81AD80AE80AF80A81
:100E400082E0C816D104E104F104E1F610925204E4
:100E500010923E0485E292E00E947A0C53C08DE32A
:100E600092E00E947A0C8091940281112DC0109220
:100E7000520410923E04C5E0D0E061E089E00E9497
:100E8000530D68EC70E080E090E00E940A0F60E093
:100E900089E00E94530D60E08CE00E94530D68ECE5
:100EA00070E080E090E00E940A0F219731F781E026
:100EB0008093940261E088E00E94530D61E070E04D
:100EC00080E090E00E940A0F1092520410923E04BB
:100ED00025C080919402882309F184E592E00E9464
:100EE0007A0CE0915204E33169F081E08E0F809337
:100EF0005204F0E0E45CFB4FC283E82FF0E0E45CD6
:100F0000FB4F128261E070E080E090E0DF91CF91D2
:100F1000FF90EF90DF90CF900C940A0FDF91CF916C
:100F2000FF90EF90DF90CF90089540918A0250910A
:100F30008B02209188023091890242175307B4F442
:100F40009091E8009570E1F39091E80092FD19C04E
:100F50008093F10080918A0290918B0201968F73A9
:100F60009927892B19F48EEF8093E80080918A02EB
:100F700090918B02019690938B0280938A0281E07C
:100F8000089580E00895615030F02091F100FC0157
:100F900020830196F8CF289884E68093090308956A
:100FA0001F920F920FB60F9211242F933F934F93DE
:100FB0005F936F937F938F939F93AF93BF93EF93C1
:100FC000FF938091B900887F803609F49CC068F552
:100FD000883209F45BC090F4803109F454C038F4CD
:100FE000882309F4F2C0883009F44DC0F2C088317A
:100FF00009F44CC0803209F45DC0EBC0803409F4C0
:1010000068C048F4803309F455C0883309F0E1C062
:1010100080933B03D4C0803509F44FC0883509F470
:101020005DC0883409F0D5C0D2C0883909F4C3C086
:10103000A8F4883709F467C038F4883609F463C027
:10104000803709F460C0C5C0883809F4B4C080395D
:1010500009F45FC0803809F0BCC05BC0803B09F474
:1010600084C038F4803A09F466C0883A09F47DC037
:10107000B0C0803C09F4A3C0883C09F4A0C0883B00
:1010800009F486C0A6C08091180310C090913A035D
:1010900080913903981770F5E0913A0381E08E0F43
:1010A00080933A03F0E0E75EFC4F80818093BB00C1
:1010B00085EC82C080933B038AC0E0913A0381E0D3
:1010C0008E0F80933A038091BB00F0E0E75EFC4F07
:1010D000808390913A03809139036AC0E0913A038A
:1010E00081E08E0F80933A038091BB00F0E0E75ED1
:1010F000FC4F808380913C03811169C081E0809323
:10110000170384EA5DC083E080933D0310920803D7
:10111000CFCF80910803803208F04DC0E0910803E2
:1011200081E08E0F809308038091BB00F0E0E851CE
:10113000FD4F8083BDCF85EC8093BC0010923D03B2
:1011400080910803803230F4E0910803F0E0E85128
:10115000FD4F10826091080370E088EE92E0E0E0BD
:10116000F0E009951092080334C084E080933D03B9
:101170001092E7021092E602E0E0F0E0099580911B
:10118000E602811105C081E08093E6021092C6025A
:10119000E091E70281E08E0F8093E702F0E0EA53EE
:1011A000FD4F80818093BB009091E7028091E60221
:1011B000981708F47DCF85E88093BC000AC085ECC1
:1011C0008093BC0010923D0304C010923B030E9428
:1011D0002E05FF91EF91BF91AF919F918F917F91DC
:1011E0006F915F914F913F912F910F900FBE0F9094
:1011F0001F9018952F923F924F925F926F927F921D
:101200008F929F92AF92BF92CF92DF92EF92FF9216
:101210000F931F93CF93DF93CDB7DEB728970FB609
:10122000F894DEBF0FBECDBFC82E962E4887190199
:1012300078010E94C3012B013C018C2C880CD12C1D
:1012400010E001E02885A22EB12CC701A0E0B0E09B
:101250008B839C83AD83BE839885D91608F089C0A3
:1012600000933E03C092600310923F03109261030B
:10127000692D82EB93E00E94B90581E00E94950BF5
:1012800000933E03C092600310923F0310926103EB
:1012900080913D038111FCCFC5018D1991098132E7
:1012A000910514F080E290E08F83813210F0A0E28B
:1012B000AF8300933D0300933C03BFEFB0933B0328
:1012C00010923A038F818150809339030093180361
:1012D0008091180388298093180380911703813027
:1012E00071F410921703809118038093BB008091D2
:1012F000BC0083FDF8CFE5ECE093BC0003C0F5EE45
:10130000F093BC0080913D038130E1F380913A037A
:101310002F81821718F430913A033F83E9E1F3E01B
:10132000A4EAB2E080E04F81841721F091919D936F
:101330008F5FF9CF1092C5024093C4028091C5021D
:101340005F81581709F444C0E114F10489F10E9447
:10135000C301DC01CB0184199509A609B7092B81CA
:101360003C814D815E8182179307A407B50700F188
:101370002FC0E114F10491F10E94C301DC01CB0103
:1013800084199509A609B7096701E12CF12C8C1580
:101390009D05AE05BF0510F14885242F30E0812F53
:1013A000012E000C990B82179307C4F41FEF16C08F
:1013B000C101810F911D17FD9A959A83898382EB54
:1013C00093E00E947005A981BA818C931F5FB6CF0C
:1013D0008885813208F080E2D80E3ECF812F289692
:1013E0000FB6F894DEBF0FBECDBFDF91CF911F9136
:1013F0000F91FF90EF90DF90CF90BF90AF909F90B4
:101400008F907F906F905F904F903F902F900895B6
:10141000BF92CF92DF92EF92FF920F931F93CF93E1
:10142000DF9300D0CDB7DEB7F82EE62EC42EB22E55
:10143000D02E08EE13E09E012E5F3F4F41E00E9448
:10144000FA08882341F14C2D50E04B1951094F5FA8
:101450005F4F81E090E002C0880F991FBA94E2F7D5
:101460000197042E01C0880F0A94EAF72D2D01C0C0
:10147000220F4A95EAF7382F30959A8193238223D9
:10148000892B8A838983AE014F5F5F4F6E2D8F2D2D
:101490000E943B0C01C080E00F900F90DF91CF9134
:1014A0001F910F91FF90EF90DF90CF90BF90089524
:1014B0008F929F92AF92BF92CF92DF92EF92FF9264
:1014C000CF93DF930E94F10BC4E6D0E0C12CD12C66
:1014D0007601460157010E94F10B6091150370914E
:1014E0001603072E000C880B990B0E94B5139B0165
:1014F000AC01C501B4010E949A124B015C016091DC
:10150000130370911403072E000C880B990B0E9493
:10151000B5139B01AC01C701B6010E949A126B0181
:101520007C012197C1F620E030E048EC52E4C5018F
:10153000B4010E940B130E947D1370939302609379
:10154000920220E030E048EC52E4C701B6010E946C
:101550000B130E947D137093910260939002DF91B0
:10156000CF91FF90EF90DF90CF90BF90AF909F9082
:101570008F9008950E947C0C8823D9F08FE692E02A
:101580000E946C0C6EEF82E693E00E94F30461E02F
:1015900089E00E94530D60E08CE00E94530D109290
:1015A000940260E088E00E94530D10928F02109226
:1015B0008E02089596E0899FD0011124A254BC4F59
:1015C00090967C936E935F9791E091969C93919700
:1015D00090912A04E0912B04F0912C04992339F086
:1015E000309751F0811108C08091DA0304C0309720
:1015F00019F05C968C910994089590E0FC01319764
:10160000EF30F105B0F5EA5AFF4F0C94591580916F
:1016100080008F7703C0809180008F7D8093800051
:10162000089580918000877FF9CF84B58F7702C0BD
:1016300084B58F7D84BD0895809190008F7707C019
:10164000809190008F7D03C080919000877F809370
:10165000900008958091C0008F7703C08091C000F2
:101660008F7D8093C00008958091C200877F809312
:10167000C20008950F931F93CF93DF93C82FD62FE7
:1016800086E0C89FF0011124E254FC4F11A2878D1F
:1016900090A181309105D9F040F082309105A9F1F7
:1016A0000397F1F560E070E034C06623C9F161E0B2
:1016B00070E08C2F0E94DA0A0E94C3016093160426
:1016C00070931704809318049093190429C00E9402
:1016D000C301009116041091170420911804309151
:1016E0001904AB01BC01401B510B620B730B8091C1
:1016F000280490912904A0E0B0E084179507A6077C
:10170000B70718F462E070E004C0D11109C063E0CB
:1017100070E08C2FDF91CF911F910F910C94DA0A1A
:10172000DF91CF911F910F910895282F3091610380
:10173000313208F04AC080913D038111FCCF909175
:10174000600342E040933D0320933C032FEF20933E
:101750003B0310923A0330933903E0E4F3E0A9E14C
:10176000B3E020E0321721F041914D932F5FFACF83
:101770001092180320911803990F922B909318033D
:1017800090911703913061F4109217039091180310
:101790009093BB009091BC0093FDF8CF95EC01C0F5
:1017A00095EE9093BC0090913D039230E1F39091BF
:1017B0003B039F3F79F080913B03803241F0809161
:1017C0003B03803331F084E005C081E003C082E058
:1017D00001C083E010923F031092610310923E0318
:1017E00008950F931F93CF93DF93CDE2D4E008EEDB
:1017F00013E02EE234E04EE06BE388810E94FA08A9
:1018000089819A8198278927982790931603809336
:1018100015038B819C81982789279827909314031F
:10182000809313038D819E81982789279827909311
:1018300012038093110389859A8598278927982711
:101840009093100380930F038B859C85982789279D
:10185000982790930E0380930D038D859E8598277E
:101860008927982790930C0380930B03DF91CF91E6
:101870001F910F910895CF93DF93EA0191E0909328
:101880003E038093600310923F031092610382EB4A
:1018900093E00E94B905688182EB93E00E94B9054C
:1018A00081E00E94950B91E0811190E0892FDF91FA
:1018B000CF910895009769F0FC0101900020E9F7AD
:1018C0003197AF01481B590BBC0182E693E00C94A1
:1018D000EC0580E090E00895CF93DF930E945A0CCE
:1018E000EC018DE092E00E945A0C8C0F9D1FDF915D
:1018F000CF9108950C945A0C80913C0490913D0432
:10190000FC01319120913E04AFE3B4E044963111E3
:1019100004C081E0222349F007C0231305C03191A0
:101920002D91E817F90799F780E008958F929F921B
:10193000AF92BF920F931F93CF93DF93CDB7DEB7D4
:10194000A1970FB6F894DEBF0FBECDBF19A24230EB
:1019500008F44AE08E010F5D1F4F842E912CA12CBC
:10196000B12CA50194010E943715E62FB901CA01D7
:1019700001501109EA3014F4E05D01C0E95CD801BE
:10198000EC93232B242B252B61F7C8010E945A0CC2
:10199000A1960FB6F894DEBF0FBECDBFDF91CF91F9
:1019A0001F910F91BF90AF909F908F9008952091BD
:1019B0000A03211103C08FEF9FEF08955FB7F894DA
:1019C00022E02093E9002091F20030E01216130685
:1019D00014F421E030E0422FFC0184E6415038F05D
:1019E0002898809309039091F1009193F7CF2115E6
:1019F000310521F08091F200882319F05FBFC90101
:101A000008958BE68093E800F9CF2FB7F89483E030
:101A10008093E9009091E800892F807295FF04C0BF
:101A20009091F20080E4891B2FBF089580915704A4
:101A300081110DC082E08093530484E080935404AC
:101A4000109256041092550481E08093570483E568
:101A500094E00895CF93DF93282F30E0F901E95502
:101A6000FE4F8491F901E857FE4FD491F901E759EF
:101A7000FE4FC491CC2391F081110E94FD0AEC2FFE
:101A8000F0E0EE0FFF1FE55AFE4FA591B491EC91E7
:101A9000ED2381E090E021F480E002C080E090E05E
:101AA000DF91CF9108951F93CF93DF93282F30E0DC
:101AB000F901E955FE4F8491F901E857FE4FD491A1
:101AC000F901E759FE4FC491CC23C1F0162F8111C3
:101AD0000E94FD0AEC2FF0E0EE0FFF1FE35BFE4FCC
:101AE000A591B4919FB7F894111104C08C91D09531
:101AF000D82302C0EC91DE2BDC939FBFDF91CF9106
:101B00001F910895CF93DF9390E0FC01E857FE4FBB
:101B10002491FC01E759FE4F8491882361F190E004
:101B2000880F991FFC01E15CFE4FC591D491FC0127
:101B3000E35BFE4FA591B491611109C09FB7F89482
:101B40008881209582238883EC912E230BC06230FC
:101B500061F49FB7F8948881322F3095832388836E
:101B6000EC912E2B2C939FBF06C08FB7F894E88181
:101B70002E2B28838FBFDF91CF9108956F927F9294
:101B80008F929F92AF92BF92CF92DF92EF92FF928D
:101B90000F931F93CF93DF9381E080932A040E94D9
:101BA000C30100911A0410911B0420911C04309170
:101BB0001D04AB01BC01401B510B620B730B8091E8
:101BC000260490912704A0E0B0E084179507A607AB
:101BD000B70708F0E6C0C0E080912404C81730F0D1
:101BE000712C812C912C5401839440C0E0912004ED
:101BF000F0912104EC0FF11D62E080810E94820DC2
:101C0000CF5FEACFC62DD0E0E0912004F09121040F
:101C1000EC0FFD1F80810E942A0D2496CC0FDD1F42
:101C2000C254DC4F892B09F04BC0888199818C29E3
:101C30009D2999838883639480912404681610F306
:101C4000E0912204F0912304E00FF11F61E0808114
:101C50000E94530D8091220490912304FC01E00F17
:101C6000F11F60E080810E94820D739480912504B1
:101C7000781658F5072D10E0E0912204F091230426
:101C8000E00FF11F61E080810E94820DE09122044B
:101C9000F0912304E00FF11F60E080810E94530D5A
:101CA000D501C401072C04C0880F991FAA1FBB1FB0
:101CB0000A94D2F76C017C01E094F094612CBCCFC3
:101CC000888199818E219F21B4CF2EEBE22E23E0D3
:101CD000F22EF7018FEF9FEF278D30A1232B21F4F8
:101CE000148E968F858F11A2369623E0EA3FF20775
:101CF00099F7C0E096E0D92E80912404C81758F5D2
:101D0000D0E00C2F10E0000F111F0A531C4F209140
:101D10002504D217F0F4F801408151810D2E02C044
:101D2000569547950A94E2F7642F6170C29F90011F
:101D300011242D0F311DEEEBF3E080E0A58DB68D63
:101D40002A173B0709F44DC08F5F36968A30B1F7EA
:101D50002CC0CF5FD1CFC0E0F70181A18111C1E0DC
:101D6000F6E0EF0EF11C2AEFE21623E0F206A1F7EF
:101D70000E94C30160931A0470931B0480931C0497
:101D800090931D04CC2369F08091DF03882349F0F0
:101D90008091DD039091DE03019719F48091DA03BD
:101DA0002AC010922A0480E026C040FF1CC0EEEB3F
:101DB000F3E080E090E0448D411117C0E0911E04F3
:101DC000F0911F04E20FF31F4081D89EF001D99ECD
:101DD000F00D1124E254FC4F448F368F258F10A252
:101DE000178E0E943A0BDF5F92CF019636968A30AB
:101DF000910509F7F8CFDF91CF911F910F91FF90D7
:101E0000EF90DF90CF90BF90AF909F908F907F909A
:101E10006F9008958F929F92AF92BF92CF92DF9270
:101E2000EF92FF926B017C010E949E014B015C01CD
:101E3000C114D104E104F104F1F00E949E01DC011F
:101E4000CB0188199909AA09BB09883E9340A105CD
:101E5000B10570F321E0C21AD108E108F10888EE5B
:101E6000880E83E0981EA11CB11CC114D104E104AA
:101E7000F10419F7DDCFFF90EF90DF90CF90BF9086
:101E8000AF909F908F900895CF93DF9300D000D0B4
:101E900000D0CDB7DEB7789484B5826084BD84B5B8
:101EA000816084BD85B5826085BD85B5816085BD55
:101EB00080916E00816080936E001092810080910D
:101EC0008100826080938100809181008160809395
:101ED00081008091800081608093800080919100DA
:101EE0008260809391008091910081608093910045
:101EF000809190008160809390008091C100846007
:101F00008093C1008091C10082608093C100809164
:101F1000C10081608093C1008091C3008160809383
:101F2000C3008091C00082608093C0008091C20095
:101F300081608093C20080917A00846080937A00EF
:101F400080917A00826080937A0080917A0081602B
:101F500080937A0080917A00806880937A00109252
:101F60000A031092960210928D028091D700816030
:101F70008093D70080EA8093D80089B5806189BDBD
:101F800089B5826089BD09B400FEFDCF61E070E0D3
:101F900080E090E00E940A0F8091D8008F7C8061E1
:101FA0008093D8008091E000807F8093E000809152
:101FB000E1008E7E8093E1008DE08093E200559AEF
:101FC000209A8FEF9FEF90936F0380936E0383E9C6
:101FD00091E00E946C0C82EA91E00E946C0C01E09E
:101FE00023E042E06BE680912D040E94080A00E0A5
:101FF00022E044E06BE180912D040E94080A22E077
:1020000044E06CE180912D040E94080AF0902D04B8
:1020100008EE13E09E012F5F3F4F41E06BE68F2DEE
:102020000E94FA0889818F7B89838A83AE014E5F83
:102030005F4F6BE68F2D0E943B0C8AEB91E00E9474
:102040006C0C9E012F5F3F4F41E065E780912D04AE
:102050000E94FA08882339F089818E7790E095955F
:10206000879580932E0480912E04843319F48BE598
:1020700091E002C089E791E00E946C0C03E022E04D
:1020800044E06CE180912D040E94080A22E044E0C3
:102090006BE180912D040E94080A809194028111C5
:1020A0000E94580A61E08CE00E94820D61E089E0A4
:1020B0000E94820D61E088E00E94820D83EC96E030
:1020C00090932C0480932B0461E089E00E94530DCF
:1020D00000E010E080919402882309F48CC10E94F2
:1020E000C3016B837C838D839E8380919702909143
:1020F0009802A0919902B0919A022B813C814D8166
:102100005E81281B390B4A0B5B0BCA01B9010E9487
:10211000B31320E030E04AE754E40E940B134B0174
:102120005C010E94F10B6091150370911603809180
:10213000920290919302681B790B072E000C880B7A
:10214000990B0E94B51320E030E040E05AE30E9472
:102150006A14A50194010E946A1423EC35EF4CE146
:1021600051E40E946A146B017C0160911303709129
:1021700014038091900290919102681B790B072EB5
:10218000000C880B990B0E94B51320E030E040E072
:102190005AE30E946A14A50194010E946A1423EC78
:1021A00035EF4CE151E40E946A144B015C01A70138
:1021B0009601C701B6010E946A146B017C01A5015A
:1021C0009401C501B4010E946A149B01AC01C701CE
:1021D000B6010E949A120E94DD1426E636E646E613
:1021E00050E40E946A146B017C0180918E029091F0
:1021F0008F0205970CF00AC188ED91E00E947A0CDD
:10220000A7019601C701B6010E941D15882319F088
:102210008FED91E01AC046015701E894B7F82FEF0F
:102220003FEF4FE75FE7C501B4010E941D15811123
:102230000FC02FEF3FEF4FE75FE7C501B4010E94EA
:10224000061318162CF483EE91E00E945A0C76C007
:102250002FEF3FEF4FE75FE4C701B6010E9465141F
:1022600018161CF487EE91E0F0CF2FEF3FEF4FE709
:102270005FECC701B6010E94061387FDF3CF20E093
:1022800030E0A901C701B6010E94061387FF09C00B
:102290006DE282E693E00E94F304C701B601905814
:1022A00002C0C701B6012AE037ED43EA5BE30E94B2
:1022B0009A122B013C010E9484134B015C010E9485
:1022C000B3139B01AC01C301B2010E9499122B010F
:1022D0003C014AE0C501B4010E94960C6EE282E620
:1022E00093E00E94F30420E030E040E251E4C301B7
:1022F000B2010E946A142B013C010E9484134B011D
:10230000A12CB12C4AE0C501B4010E94960CC50174
:10231000B4010E94B3139B01AC01C301B2010E943E
:10232000991220E030E040E251E40E946A140E94D9
:10233000841380E090E04AE00E94960C8BEE91E0DE
:102340000E947A0C20E030E040EC5FE3C701B60168
:102350000E94651418164CF480918E0290918F02A1
:10236000019690938F0280938E0280918E029091BD
:102370008F02059764F181EF91E00E947A0C61E091
:1023800089E00E94530D60E088E00E94530D61E0F7
:102390008CE00E94530D6AE070E080E090E00E94C3
:1023A0000A0F0E94BE0D0E94BA0A60E089E00E94F6
:1023B000530D61E088E00E94530D60E08CE00E94C4
:1023C000530D6AE070E080E090E00E940A0F8B817C
:1023D0009C81AD81BE818093970290939802A093D7
:1023E0009902B0939A0265E070E080E090E00E946C
:1023F0000A0F0E94580A0E94BE0D0E94BA0A0115D7
:10240000110509F467CE0E94000064CE20E030E0A0
:1024100040EC5FE3C701B6010E94651418160CF486
:102420009BCFA9CF109265031092640388EE93E0CE
:10243000A0E0B0E08093660390936703A0936803E5
:10244000B093690321E331E0309363032093620387
:102450002FEF3FEF30936F0320936E031092B5037D
:102460001092B4038093B6039093B703A093B8037C
:10247000B093B90383E491E09093B3038093B203E4
:1024800083E892E090933D0480933C0410925204C0
:1024900010923E0488E680932D041092C00310929F
:1024A000C4031092C3031092C50385E591E0909395
:1024B000BF038093BE03EEEBF3E08AEF93E0148E4C
:1024C00010A2178E11A236968E179F07C1F780E1D2
:1024D00091E090932104809320048CE091E090930C
:1024E00023048093220484E08093240480932504B1
:1024F00084E191E090931F0480931E048AE090E0B1
:10250000909327048093260484EF91E0909329040C
:102510008093280410922C0410922B0410921A0419
:1025200010921B0410921C0410921D0410922A0495
:1025300008955058BB27AA270E94B1120C942B145F
:102540000E941D1438F00E94241420F039F49F3F9B
:1025500019F426F40C941A140EF4E095E7FB0C948D
:102560001414E92F0E943C1458F3BA17620773073A
:102570008407950720F079F4A6F50C945E140EF408
:10258000E0950B2EBA2FA02D0B01B90190010C0183
:10259000CA01A0011124FF27591B99F0593F50F49B
:1025A000503E68F11A16F040A22F232F342F4427F3
:1025B000585FF3CF469537952795A795F0405395EB
:1025C000C9F77EF41F16BA0B620B730B840BBAF0BB
:1025D0009150A1F0FF0FBB1F661F771F881FC2F726
:1025E0000EC0BA0F621F731F841F48F4879577953A
:1025F0006795B795F7959E3F08F0B0CF9395880FF4
:1026000008F09927EE0F9795879508950E94F0138B
:1026100008F481E008950E941F130C942B140E946B
:10262000241458F00E941D1440F029F45F3F29F053
:102630000C94141451110C945F140C941A140E94ED
:102640003C1468F39923B1F3552391F3951B550B73
:10265000BB27AA2762177307840738F09F5F5F4F75
:10266000220F331F441FAA1FA9F335D00E2E3AF0B4
:10267000E0E832D091505040E695001CCAF72BD0CC
:10268000FE2F29D0660F771F881FBB1F261737071D
:102690004807AB07B0E809F0BB0B802DBF01FF274F
:1026A00093585F4F3AF09E3F510578F00C94141404
:1026B0000C945F145F3FE4F3983ED4F386957795CE
:1026C0006795B795F7959F5FC9F7880F911D969508
:1026D000879597F90895E1E0660F771F881FBB1F64
:1026E000621773078407BA0720F0621B730B840B11
:1026F000BA0BEE1F88F7E09508950E948413689442
:10270000B1110C945F1408950E94441488F09F57EF
:1027100098F0B92F9927B751B0F0E1F0660F771F05
:10272000881F991F1AF0BA95C9F714C0B13091F0FB
:102730000E945E14B1E008950C945E14672F782F08
:102740008827B85F39F0B93FCCF3869577956795C0
:10275000B395D9F73EF490958095709561957F4F2C
:102760008F4F9F4F0895E89409C097FB3EF49095D2
:102770008095709561957F4F8F4F9F4F9923A9F05A
:10278000F92F96E9BB279395F695879577956795E9
:10279000B795F111F8CFFAF4BB0F11F460FF1BC02D
:1027A0006F5F7F4F8F4F9F4F16C0882311F096E9C0
:1027B00011C0772321F09EE8872F762F05C066236E
:1027C00071F096E8862F70E060E02AF09A95660F27
:1027D000771F881FDAF7880F9695879597F90895E0
:1027E000990F0008550FAA0BE0E8FEEF1616170622
:1027F000E807F907C0F012161306E407F50798F08A
:10280000621B730B840B950B39F40A2661F0232BA2
:10281000242B252B21F408950A2609F4A140A6951E
:102820008FEF811D811D089597F99F6780E870E003
:1028300060E008959FEF80EC089500240A94161636
:10284000170618060906089500240A94121613069E
:10285000140605060895092E0394000C11F488232C
:1028600052F0BB0F40F4BF2B11F460FF04C06F5F48
:102870007F4F8F4F9F4F089557FD9058440F551F1E
:1028800059F05F3F71F04795880F97FB991F61F0F2
:102890009F3F79F087950895121613061406551F69
:1028A000F2CF4695F1DF08C0161617061806991FD5
:1028B000F1CF86957105610508940895E894BB27CA
:1028C00066277727CB0197F908950E94F01308F443
:1028D0008FEF08950E947D140C942B140E941D14F8
:1028E00038F00E94241420F0952311F00C94141455
:1028F0000C941A1411240C945F140E943C1470F36D
:10290000959FC1F3950F50E0551F629FF001729F94
:10291000BB27F00DB11D639FAA27F00DB11DAA1FA3
:10292000649F6627B00DA11D661F829F2227B00DF0
:10293000A11D621F739FB00DA11D621F839FA00D7B
:10294000611D221F749F3327A00D611D231F849FCB
:10295000600D211D822F762F6A2F11249F57504022
:102960009AF0F1F088234AF0EE0FFF1FBB1F661F9D
:10297000771F881F91505040A9F79E3F510580F066
:102980000C9414140C945F145F3FE4F3983ED4F35A
:10299000869577956795B795F795E7959F5FC1F70A
:1029A000FE2B880F911D9695879597F9089519F438
:1029B00016F40C941A140C9422150E944414B8F3C3
:1029C0009923C9F3B6F39F57550B87FF0E94301523
:1029D0000024A0E640EA900180585695979528F487
:1029E000805C660F771F881F20F02617370748077F
:1029F00030F4621B730B840B202931294A2BA695D6
:102A000017940794202531254A2758F7660F771F1A
:102A1000881F20F026173707480730F4620B730B26
:102A2000840B200D311D411DA09581F7B901842F24
:102A30009158880F9695879508950E94F013880BFA
:102A4000990B08959F3F31F0915020F48795779529
:102A50006795B795880F911D9695879597F9089575
:102A600091505040660F771F881FD2F70895A1E25A
:102A70001A2EAA1BBB1BFD010DC0AA1FBB1FEE1FF8
:102A8000FF1FA217B307E407F50720F0A21BB30B43
:102A9000E40BF50B661F771F881F991F1A9469F7BF
:102AA00060957095809590959B01AC01BD01CF011B
:102AB0000895EE0FFF1F0590F491E02D099481E039
:0C2AC00090E0F8940C946415F894FFCF9B
:102ACC00FFFFFFFF00E10000000000000706050407
:102ADC000302010031323341343536423738394341
:102AEC002A30234400C18081000000E8030000006C
:102AFC0000F304EC057206090514059A0676060027
:102B0C00000000B9058C05E90560058405700561B8
:102B1C000500000000BF06BB06B8064D5055363008
:102B2C00353020636F6E6E656374696F6E207375DC
:102B3C00636365737366756C004D50553630353074
:102B4C0020636F6E6E656374696F6E206661696C6D
:102B5C00656400426567696E2073657475702E2E0E
:102B6C002E00696E697469616C697A696E67204DB3
:102B7C005055363035302E2E2E0074657374696EB8
:102B8C0067204D50553630353020636F6E6E65635F
:102B9C0074696F6E2E2E2E000976656C3A20006ECD
:102BAC00616E00696E66006F7666006B6D2F682C27
:102BBC0000414C41524D20495320545249474745FE
:102BCC005245442100456E7465723A20000D0A008E
:102BDC00232028706F756E642920697320707265CC
:102BEC00737365640070617373776F726420696EC0
:102BFC00707574206973207265736574002A2028BF
:102C0C0061737465726978292069732070726573B9
:102C1C007365640061206E756D6265722028302EBC
:102C2C002E39292069732070726573736564007086
:102C3C00617373776F726420697320636F7272654E
:082C4C006374003935303300D8
:2070000055C000006EC000006CC000006AC0000068C0000066C0000064C0000062C0000043
:2070200060C000005EC00000F2C400005AC0000058C0000056C0000054C0000052C00000EE
:2070400050C0000078C000004CC000004AC0000048C0000046C0000044C0000042C00000BE
:2070600040C000003EC000003CC000003AC0000038C0000036C0000034C0000032C0000048
:2070800030C000002EC000002CC000002AC0000028C0000026C0000024C0000022C00000A8
:2070A00020C000001EC000001CC0000011241FBECFEFDAE0DEBFCDBF11E0A0E0B1E0E2E3BC
:2070C000FFE702C005900D92A83AB107D9F711E0A8EAB1E001C01D92AE3BB107E1F78FD30B
:2070E00026C78ECFF89410926F0010928100109285001092840081E085BF15BE47985D9AEB
:20710000289A0C94000008952091B2013091B3012F5F3F4F3093B3012093B201932F37FFA6
:2071200003C08EEF831B982F990F921710F447980895479A08951F920F920FB60F9211246E
:207140002F938F939F93EF93FF9310928500109284008091A8019091A901009741F00197D3
:207160009093A9018093A801892B09F45D9A8091AA019091AB01009741F001979093AB0126
:207180008093AA01892B09F4289AE0E0F0E0859194918F5F9F4F49F08091AC019091AD0151
:2071A00001969093AD018093AC01FF91EF919F918F912F910F900FBE0F901F90189584E0BC
:2071C0008093E9000DC08091E8008B778093E80003C08EB3882351F08091E80082FFF9CFBE
:2071E0008091E80085FFEFCF8091F1000895982F83E08093E9008091E80085FD0DC0809136
:20720000E8008E778093E80003C08EB3882369F08091E80080FFF9CF9093F1005D9884E6CB
:2072200090E09093A9018093A80108954F925F926F927F928F929F92AF92BF92CF92DF921E
:20724000EF92FF920F931F93CF93DF9384E08093E9008091E80082FF57C2289884E690E067
:207260009093AB018093AA01AADF182F853481F48CE49DE19093AD018093AC0107B600FC4B
:20728000FDCFF999FECF81E180935700E89503C0843519F494DF8DE00DC28C34E1F38035F9
:2072A000D1F3843721F484E4A2DF80E003C2813611F489E5FFC18134B1F481DF182F7FDFE3
:2072C00090E0880F991FAA2797FDA095BA2F312F330F20E0442737FD4095542F822B932B68
:2072E000A42BB52BB8C1803711F483E5E3C1833549F4C0E0D1E089917ADF21E0C730D20714
:20730000D1F7D9C1863521F481E371DF80E3D2C1833731F487E86BDF85E969DF8EE1CAC149
:207320008536B9F4E0E0F0E093E085E090935700E89507B600FCFDCF80935700E89507B65D
:2073400000FCFDCFE058FF4FA0E7E030FA0771F7A2CF823739F4E1E0F0E089E08093570024
:207360008491A8C1863439F4E0E0F0E089E08093570084919FC18E3439F4E3E0F0E089E0E5
:2073800080935700849196C1813539F4E2E0F0E089E08093570084918DC1823631F489E521
:2073A00026DF80E024DF80E885C1823419F0873609F0E5C01092AD011092AC0100DF082FE8
:2073C000FEDEF82EFCDE682E8554823008F071C1902F80E0CF2DD0E0C82BD92B10926F00B3
:2073E000173609F04BC081E180935700E895DD24CC24C3943FC0E090AE01F090AF010091CC
:20740000B0011091B101B6E46B16D9F4ED2DF0E0EE29FF29E4918E2FEADEDD2081F082E08D
:2074200090E0A0E0B0E0E80EF91E0A1F1B1FE092AE01F092AF010093B0011093B101DC2470
:2074400018C0D801C701B695A7959795879559D5CEDE82E090E0A0E0B0E0E80EF91E0A1FF2
:207460001B1FE092AE01F092AF010093B0011093B1012197209709F0BECF7DC08090AE01F5
:207480009090AF01A090B001B090B10196E4691609F05DC083E0F40180935700E89507B63E
:2074A00000FCFDCF54C0F6E46F1661F5772031F1E090AE01F090AF010091B0011091B1019E
:2074C0007EDED82ECC24852D90E08C299D29F7010C0140925700E895112482E090E0A0E08B
:2074E000B0E0E80EF91E0A1F1B1FE092AE01F092AF010093B0011093B10102C060DE582E1A
:20750000742423C0E090AE01F090AF010091B0011091B10116950795F794E79450DE682FFA
:20752000C701F7D48091AE019091AF01A091B001B091B1010296A11DB11D8093AE01909349
:20754000AF01A093B001B093B101219704C05524772444244394209709F0A5CF96E46916B6
:2075600041F485E0F40180935700E89507B600FCFDCF8DE03CDE82E080936F009CC0833492
:2075800071F40091AE011091AF0119DE90E021E0F8010C0120935700E89511247CCE8336C8
:2075A00019F5E090AE01F090AF010091B0011091B10105DEF701E16090E021E00C0120938C
:2075C0005700E895112482E090E0A0E0B0E0E80EF91E0A1F1B1FE092AE01F092AF0100936A
:2075E000B0011093B10157CE8D3661F4E091AE01F091AF0185E080935700E89507B600FCF2
:20760000FDCF49CE823551F4E091AE01F091AF0105911491812FEBDD802F4CC0843421F5FE
:20762000E090AE01F090AF010091B0011091B10116950795F794E794C2DD682FC70169D4DE
:207640008091AE019091AF01A091B001B091B1010296A11DB11D8093AE019093AF01A093D8
:20766000B001B093B10117CE843609F5E090AE01F090AF010091B0011091B101D801C70142
:20768000B695A795979587953CD4B1DD82E090E0A0E0B0E0E80EF91E0A1F1B1FE092AE010A
:2076A000F092AF010093B0011093B10104C08B3111F08FE39CDD83E08093E9009091E8002B
:2076C0008091E8008E778093E80095FF04C010C08EB38823C9F08091E80080FFF9CF809193
:2076E000E8008E778093E80003C08EB3882361F08091E80080FFF9CF84E08093E9008091F1
:20770000E8008B778093E800DF91CF911F910F91FF90EF90DF90CF90BF90AF909F908F90AC
:207720007F906F905F904F9008959091B601892F8F77813249F58091B7018032A1F081328A
:2077400019F5913A09F58091E800877F8093E8008DE091E067E070E00BD28091E8008B770B
:207760008093E8000895913279F48091E800877F8093E8008DE091E067E070E05DD2809192
:20778000E8008E778093E800089582E061EC42E0B5D083E061E842E1B1D084E060E842E1EF
:2077A000ADC084B7877F84BF88E10FB6F89480936000109260000FBE20E880E090E00FB63F
:2077C000F89420936100809361000FBE81E085BF92E095BF3F9A209A559AE1E6F0E02083A1
:2077E000108247985D9A289A109289008AEF8093880090936F0083E080938100F0C0409116
:20780000000850910108109201081092000894B714BE88E10FB6F8948093600010926000D5
:207820000FBE292F30E0F901E270F07091FD18C090FF05C0859194918F5F9F4F81F423FFFF
:207840000FC08091090190910A014817590741F0E0E0F0E0859194918F5F9F4F09F042DC64
:20786000A0DF78941092AD011092AC010CC0DEDC36D38091AC019091AD0181549F4110F00D
:207880001092140141DC80911401882381F78091E00081608093E00025DC80E090E0089598
:2078A000FA01923049F0933061F09130F9F485E191E022E130E01EC087E291E02EE330E04D
:2078C00019C0882329F485E691E024E030E012C0813029F489E691E022E230E00BC0823006
:2078E00029F48DE891E028E130E004C080E090E020E030E091838083C90108958093E9004E
:207900008091EB0081608093EB001092ED006093EC004093ED008091EE00881F8827881F62
:2079200008958091B60188238CF403C08EB38823B1F08091E80082FFF9CF8091E8008B772A
:207940008093E80008958EB3882349F08091E80080FFF9CF8091E8008E778093E800089594
:20796000EF92FF920F931F9345D04CD008ED10E0F80180818F77808380818068808380819B
:207980008F7D808319BC1EBA1092B40180EEE82EF12CF70180818B7F8083F8018081816052
:2079A000808380E060E042E0A9DFE1EEF0E080818E7F8083E2EEF0E0808181608083808144
:2079C00088608083F70180818E7F8083F8018081806180831F910F91FF90EF900895E7ED06
:2079E000F0E08081816080838AE482BF81E08093B501B6CFE8EDF0E080818E7F808310921C
:207A0000E20008951092DA001092E10008951F920F920FB60F9211242F933F934F935F93F6
:207A20006F937F938F939F93AF93BF93EF93FF938091DA0080FF1BC08091D80080FF17C0B2
:207A40008091DA008E7F8093DA008091D90080FF0BC080E189BD82E189BD09B400FEFDCF36
:207A600081E08EBB3BD203C019BC1EBA37D28091E10080FF17C08091E20080FF13C0809138
:207A8000E2008E7F8093E2008091E20080618093E2008091D80080628093D80019BC85E049
:207AA0008EBB1CD28091E10084FF2CC08091E20084FF28C080E189BD82E189BD09B400FEC5
:207AC000FDCF8091D8008F7D8093D8008091E1008F7E8093E1008091E2008F7E8093E20012
:207AE0008091E20081608093E2008091B401882331F48091E30087FD02C081E001C084E067
:207B00008EBBECD18091E10083FF21C08091E20083FF1DC08091E100877F8093E10082E06A
:207B20008EBB1092B4018091E1008E7F8093E1008091E2008E7F8093E2008091E2008061E9
:207B40008093E20080E060E042E0D8DEC7D1FF91EF91BF91AF919F918F917F916F915F9130
:207B60004F913F912F910F900FBE0F901F9018959C014091BC015091BD014617570718F49D
:207B8000F90190E044C06115710511F0AB01F8CF8091E8008E778093E80040E050E0F0CF0F
:207BA0008EB3882309F444C0853009F443C08091E80083FF02C081E008958091E80082FD70
:207BC00031C08091E80080FF22C08091F3009091F200782F60E0292F30E0262B372B07C07A
:207BE00081918093F100415050402F5F3F4F4115510519F02830310598F390E02830310566
:207C000009F491E08091E8008E778093E8004115510531F6992321F605C08EB3882341F075
:207C2000853041F08091E80082FFF7CF80E0089582E0089583E008959C016115710529F47C
:207C40008091E8008B778093E800F90126C08EB3882391F1853091F18091E80083FF02C06C
:207C600081E008958091E80082FFF1CF06C08091F10081936150704059F02091F300809191
:207C8000F200322F20E090E0822B932B892B79F78091E8008B778093E80061157105B9F601
:207CA00005C08EB3882341F0853041F08091E80080FFF7CF80E0089582E0089583E00895C2
:207CC0000F931F93DF93CF9300D0CDB7DEB7E6EBF1E08091F100819381E0EE3BF807C9F792
:207CE00024DD8091E80083FFE4C08091B6019091B701953009F46DC0963040F4913081F1A7
:207D0000913070F0933009F0D4C02AC0983009F4A3C0993009F4B2C0963009F0CAC07CC023
:207D2000803809F4C6C0823809F0C3C08091BA0187708093E9008091EB001092E9002091DB
:207D4000E800277F2093E80090E025E0969587952A95E1F781708093F1001092F10087C0D8
:207D6000882319F0823009F0A4C08F71823009F0A0C08091B801882331F52091BA01277097
:207D800009F497C02093E9008091EB0080FF1BC0933021F48091EB00806213C08091EB0018
:207DA00080618093EB0081E090E002C0880F991F2A95E2F78093EA001092EA008091EB00E5
:207DC00088608093EB001092E9008091E800877F51C0882309F06DC01091B8011F770FB79B
:207DE000F8948091E800877F8093E8009ADD8091E80080FFFCCF8091E3008078812B809398
:207E0000E30080688093E300112311F482E001C083E08EBB0FBF4DC08058823008F049C033
:207E20008091B8019091B9016091BA01AE014F5F5F4F36DDBC01009709F43BC08091E8008E
:207E4000877F8093E80089819A8192DE8091E8008B778093E8002DC0803859F58091E800AA
:207E6000877F8093E8008091B4018093F1008091E8008E778093E80054DD1BC08823C9F4CA
:207E80009091B8019230A8F48091E800877F8093E8009093B40145DD8091B401882331F420
:207EA0008091E30087FD02C081E001C084E08EBB6CDC8091E80083FF0AC08091EB0080624E
:207EC0008093EB008091E800877F8093E8000F900F90CF91DF911F910F91089508951F9360
:207EE0008EB3882361F01091E9001092E9008091E80083FF01C0E4DE17701093E9001F916F
:207F00000895F999FECF92BD81BDF89A992780B50895262FF999FECF1FBA92BD81BD20BDBD
:207F20000FB6F894FA9AF99A0FBE01960895F894FFCF4341544552494E4100777700080031
:207F40000000000000080112011001020000084123360001000201000109023E00020100FF
:207F600080320904000001020201000524001001042402040524060001070582030800FF0C
:207F800009040100020A000000070504021000010705830210000104030904220341007216
:207FA000006400750069006E006F0020004C0065006F006E006100720064006F0000001836
:1A7FC00003410072006400750069006E006F0020004C004C004300000000D7
:00000001FF
